:020000040800F2
:10000000301B0020E10200086D3100089D2F000820
:1000100069310008FD0F00080538000800000000E5
:100020000000000000000000000000001532000881
:100030008D1C0008000000009D31000849320008B6
:10004000FB020008FB020008FB020008FB0200089C
:10005000FB020008FB020008FB020008FB0200088C
:10006000FB020008FB020008FB020008FB0200087C
:10007000FB020008FB020008FB020008FB0200086C
:10008000FB020008FB020008FB020008FB0200085C
:10009000FB020008FB020008FB020008FB0200084C
:1000A000FB020008FB020008FB020008FB0200083C
:1000B000FB02000809330008FB020008FB020008ED
:1000C000FB020008FB020008FB020008FB0200081C
:1000D000FB020008E1370008F1370008FB020008C6
:1000E000FB020008FB020008FB020008FB020008FC
:1000F000FB020008FB020008FB020008FB020008EC
:10010000FB020008FB020008FB020008FB020008DB
:10011000FB020008FB020008FB020008FB020008CB
:10012000FB020008FB020008FB020008FB020008BB
:10013000FB020008FB020008FB020008FB020008AB
:10014000FB020008FB020008FB020008FB0200089B
:10015000FB020008FB020008FB020008FB0200088B
:10016000FB020008FB020008FB020008FB0200087B
:10017000FB020008FB020008FB0200080000000070
:10018000FB020008FB02000800F002F800F098F8FB
:100190000AA090E8000C82448344AAF10107DA45E2
:1001A00001D100F08DF8AFF2090EBAE80F0013F09C
:1001B000010F18BFFB1A43F001031847B06100009C
:1001C000D0610000103A24BF78C878C1FAD852072D
:1001D00024BF30C830C144BF04680C6070470000C1
:1001E0000023002400250026103A28BF78C1FBD840
:1001F000520728BF30C148BF0B6070476E2900F01E
:10020000D985702900F02F82662905F0CE866529F0
:1002100005F0CB86672905F0C886612905F0C786F9
:1002200003681B0A28BF41F08001692900F0A08102
:10023000642900F09D81752900F09A816F2900F0F2
:100240000D87782900F0FB81E92900F07386E42905
:1002500000F07086F52900F06D86EF2900F00A871E
:10026000F82900F0FA810368DB0928BF41F080011A
:10027000632900F0E285732900F0E785E32901F0A6
:100280003183F32901F03683002070471FB505F054
:100290007FFE9DE8030000F0C5FC00F0A3FC040015
:1002A0000020002105F048FE401C60600020002175
:1002B00005F058FEE06000F07DFC1FBD10B510BDDC
:1002C00001F096FB1146FFF7E1FF03F06FFF01F02D
:1002D00075FC03B4FFF7F2FF03BC03F0FDFA000066
:1002E0000948804709480047FEE7FEE7FEE7FEE7CA
:1002F000FEE7FEE7FEE7FEE7FEE7FEE70448054906
:10030000054A064B70470000F532000889010008D5
:1003100030150020301B002030170020301700203F
:100320007047000010B500F05DFC001D10BD00BF5F
:10033000095C000070B5064600F050FC056806F147
:100340000B0020F00704B4429CBF002070BD2B4678
:100350006A68BAB11068A04210D304F1080188425B
:100360003CBF5068586007D351681019416011684C
:10037000091B016058601460101D70BD134652685F
:10038000002AE7D12146284600F038FC0028DED1BB
:1003900070BD70B50446051F00F020FC0068002CFD
:1003A00014BF446870BD002C18BFAC423CBF20464F
:1003B0006468F8D301680A18AA4218BF456003D1DF
:1003C0002A6805461144016028684119A1421CBFF2
:1003D0006C6070BD6168696021680844286070BD08
:1003E00053EA020C00F069802DE9F04B4FF0000653
:1003F000002B1FBFB3FA83F503FA05F424FA05F6C0
:100400005E4012BF1643B2FA82F502FA05F4C5F156
:1004100020051EBF22FA05FC44EA0C04203556EAEA
:10042000044C4FEA144418BF641C4FF000084FF00E
:100430000009904271EB030C39D3002919BFB1FABE
:1004400081F701FA07F6B0FA80F700FA07F6C7F16C
:1004500020071EBF20FA07FC46EA0C062037B6FB31
:10046000F4FCA7EB0507103F07F01F0BCBF12006AC
:100470002CFA06F60CFA0BFB44BFB3460026202FDD
:10048000A4BF5E464FF0000B5BEA060C08BF4FF0BE
:10049000010B19EB0B0948EB0608ABFB027C06FBD2
:1004A00002CC0BFB03CCC01B71EB0C01C1E70B466C
:1004B000024641464846BDE8F08B13B5084318BFD5
:1004C0004FF0FF300146AFF30080BDE81C4070479D
:1004D0007CB51D4616460C00009001D02044401EFD
:1004E000074B7B442A4669460190304600F07BFC6E
:1004F00005461CB10020694600F088FC28467CBDFA
:10050000310900000FB4044910B503AA029800F0A5
:10051000A1FC10BC5DF814FB8400002070B50C46F3
:100520000546012A05D02878800600D5EA6900230F
:1005300002E0012305E05B1C934202D2E05C00284C
:10054000F9D1A869E618C01AA861286A1844286277
:10055000284600F09DFB04E0D5E9012114F8010BC9
:100560009047B442F8D3284600F0A8FB70BD0000C5
:100570002DE9F0410646002410687529314616A57C
:1005800010D000F0ACFB002802DA404213A507E0CF
:1005900031688A0701D512A502E0490704D511A5E3
:1005A000012401E000F0A4FB00210A2206F1240747
:1005B00009E0B0FBF2FCB0FBF2F302FB1C003030B0
:1005C00078541846491C0028F3D123462A46304661
:1005D000BDE8F04100F095BB000000002D000000D8
:1005E0002B00000020000000F0B40D460188090532
:1005F00002D5214C7C4402E01F4C7C440E34002187
:1006000000F1240608E002F00F071209E75D42EA54
:1006100003721B097754491C52EA0307F3D102788D
:100620000023120704D5702D06D009B1022311341E
:100630002246F0BC00F065BB01231034F8E770B52A
:1006400004460D462146106800F052FB024629463A
:100650002046BDE870400023C6E7D21D22F0070304
:10066000D3E90023C0E70368126843F02003036066
:100670000823C3610023B7E7BA5900002DE9F05FF2
:10068000894604464FF0000ADFF874B1FB44C0F815
:1006900020A02046E1688847002874D0252806D08D
:1006A000D4E901219047206A401C2062F1E700262E
:1006B0005F462046E16888472028054607DB312D44
:1006C00005D2781910F8200C08B10643F1E7B007FD
:1006D00001D526F00406C4F81CA00027C4F818A011
:1006E0002A2D09D0284605F01FFC38B304EB8708F3
:1006F000303DC8F8185019E059F8041B204604EBA7
:1007000087029161E1688847012F054618D1E069A9
:10071000002820DA26F020061DE0D8F8180000EBAB
:10072000800005EB40003038C8F818002046E1682A
:100730008847054605F0F8FB0028EED1012F0AD0C6
:100740002E2D08D12046E16888477F1C0546022FE0
:1007500046F02006C4DBA069002803DA404246F0D8
:100760000106A061F00701D026F010066C2D0BD019
:10077000682D09D04C2D39D06A2D35D0742D35D047
:100780007A2D33D016E038E0E1682F4620468847BE
:10079000B842054609D16C2F26D04FF48060E1683D
:1007A000064320468847054604E06C2F1AD04FF4D4
:1007B000807006430DB3A5F14100192802D82035F9
:1007C00046F400664A462946204626604E46FFF714
:1007D00015FD80B101280BD0F61D26F0070000F1B1
:1007E000080956E74020E4E78020D8E70020D6E754
:1007F00006F104094DE7284652E7206ABDE8F09F5C
:100800004A59000070B5064600F0F0F90468054644
:1008100030460A22002100F037FC2C6070BD000039
:1008200010B5044603E003F029FC401C09D014F87D
:10083000010B05490028F6D1BDE810400A2003F05D
:100840001DBC4FF0FF3010BD840000200EB50546E2
:1008500014460E4613A000F0B6FB284600F0B3FB8A
:1008600016A000F0B0FB304600F0ADFB15A000F084
:10087000AAFB00218DF80B100A210DF10A008DF85A
:100880000A1008E094FBF1F201FB124294FBF1F430
:10089000303200F8012D002CF4DC00F094FB00F065
:1008A00087FB00002A2A2A20617373657274696FBE
:1008B0006E206661696C65643A2000002C206669D0
:1008C0006C6520002C206C696E65200040EA0103F5
:1008D00010B59B070FD1042A0DD310C808C9121FE9
:1008E0009C42F8D020BA19BA884201D9012010BD23
:1008F0004FF0FF3010BD1AB1D30703D0521C07E0F0
:10090000002010BD10F8013B11F8014B1B1B07D153
:1009100010F8013B11F8014B1B1B01D1921EF1D1C4
:10092000184610BD40EA0103024630B59B0710D1BE
:100930004FF0013400E008C208C91D1B9D4315EAB1
:10094000C41FF8D013F0FF0102F8011B0DD01B0AE1
:10095000F8E711F8013B002B02F8013B05D011F834
:10096000013B002B02F8013BF3D130BD10B5431C15
:1009700002E010F8011B71B18107FAD14FF001328A
:1009800002C88C1A8C4314EAC211F9D0C01A0A06A4
:1009900003D0C01E10BDC01A10BD0A0401D0801EB5
:1009A00010BD0902FCD0401E10BD032A40F2308069
:1009B00010F0030C00F0158011F8013BBCF1020FA0
:1009C000624498BF11F801CB00F8013B38BF11F821
:1009D000013BA2F1040298BF00F801CB38BF00F838
:1009E000013B11F0030300F02580083AC0F00880B5
:1009F00051F8043B083A51F804CBA0E80810F5E799
:100A0000121D5CBF51F8043B40F8043BAFF300807B
:100A1000D20724BF11F8013B11F801CB48BF11F8F0
:100A2000012B24BF00F8013B00F801CB48BF00F8C0
:100A3000012B704710B5203AC0F00B80B1E8185078
:100A4000A0E81850B1E81850A0E81850203ABFF4B8
:100A5000F5AF5FEA027C24BFB1E81850A0E8185057
:100A600044BF18C918C0BDE810405FEA827C24BFAB
:100A700051F8043B40F8043B08BF7047D20728BF39
:100A800031F8023B48BF11F8012B28BF20F8023B88
:100A900048BF00F8012B70474FF000020429C0F056
:100AA000128010F0030C00F01B80CCF1040CBCF1A0
:100AB000020F18BF00F8012BA8BF20F8022BA1EBF2
:100AC0000C0100F00DB85FEAC17C24BF00F8012BD7
:100AD00000F8012B48BF00F8012B70474FF00002CF
:100AE00000B5134694469646203922BFA0E80C5024
:100AF000A0E80C50B1F12001BFF4F7AF090728BFFF
:100B0000A0E80C5048BF0CC05DF804EB890028BF7A
:100B100040F8042B08BF704748BF20F8022B11F0A3
:100B2000804F18BF00F8012B704700000000000044
:100B300030B44FF0013C50F8042B51F8043BCCFA90
:100B400052F4D51A20D1FCB950F8042B51F8043BCB
:100B5000CCFA52F4D51A17D1B4B950F8042B51F885
:100B6000043BCCFA52F4D51A0ED16CB950F8042BD0
:100B700051F8043BCCFA52F4D51A05D1002CDAD046
:100B800030BC4FF00000704729BAB1FA81F111F082
:100B90001801D1F120008440F2D1CA40CB4012F0BC
:100BA000FF0213F0FF0330BCD01A70477047704744
:100BB0007047000070B5064C7C44064D7D4404E04F
:100BC0002046016808448047241DAC42F8D170BD1E
:100BD000FC580000FC5800007047000000487047B7
:100BE000280000200048704740000020004870475F
:100BF00020000020704770477047704738B50446A2
:100C00000A4600206946AFF30080002808BF38BDBF
:100C100002460099204600F06FFA012038BD0120FD
:100C200000F0DFBEF8B5AFF30080054600200C46AB
:100C3000102000BF0646A819A0420DD932466946C9
:100C40000020AFF30080070008BF00F0CAFE009844
:100C5000A04218BF0546C419FFF7C0FF056007464C
:100C6000F01D20F007004619284600F00AF8B442AB
:100C700008BFF8BDA21B31463868BDE8F84000F057
:100C80003BBA00210160C0E9011070471020704795
:100C900070B5044685690068C10601D5302600E0BC
:100CA0002026C00707D070BDD4E901213046904707
:100CB000206A401C20626D1EF6D570BD70B50446DA
:100CC00085690078C00707D170BDD4E901212020D3
:100CD0009047206A401C20626D1EF6D570BD0968E1
:100CE0004A0501D540B27047C905FCD500B270472E
:100CF00009684A0501D5C0B27047C905FCD580B264
:100D000070472DE9F0470D4699469246044600F19A
:100D100024080168880604D5E06921F010012160EB
:100D200000E00120A84201DD471B00E00027A16987
:100D30007A1902EB0900081AA0612078C00602D4D3
:100D40002046FFF7A5FF002608E0D4E901211AF8A4
:100D500006009047206A401C761C20624E45F4DB5A
:100D60002078C0060AD52046FFF792FF06E0D4E9B6
:100D7000012130209047206A401C2062381EA7F1D4
:100D80000107F4DC07E0D4E9012118F805009047D9
:100D9000206A401C2062281EA5F10105F3DC2046D4
:100DA000FFF78CFF2078000602D50220BDE8F0870F
:100DB0000120FBE711680268006A530501D508703D
:100DC0000AE0D30501D5088006E0130603D5C21753
:100DD000C1E9000200E008600120704701694A1C77
:100DE00002610878704700B58FB0CDE9013100216C
:100DF000059105497944CDE9031011466846FFF78E
:100E00003DFC0FB000BD0000E5FFFFFF0A6802F8DF
:100E1000010B0A607047D1E900239A4202D2531CA9
:100E20000B601070704710B5436913B1AFF30080C9
:100E300001E0FFF773FB012010BD127800F12401DF
:100E40000A7000224A700122EDE711684FF0FF326C
:100E5000E9E70000074B70B50D467B44FFF7C3FF81
:100E60000446284600F0BEF810B14FF0FF3070BDC8
:100E7000204670BD1F3200002DE9FF5F15468A46EF
:100E80000446DFF8AC80F8440027D8E900103E465D
:100E9000CDE9001010E03AF816106A4602A800F0FA
:100EA0007CFD411C07D02178890603D5E2693918F9
:100EB00091420DD80744761C2078800602D5E0695F
:100EC000B84205DDAE42E6DB3AF816000028E2D172
:100ED000A069C01BA0612046FFF7DAFED8E9001028
:100EE000CDE90010002017E03AF818106A4602A871
:100EF00000F053FDB0F1FF3F81460BD000250DF10E
:100F0000080B05E0D4E901211BF8050090476D1C92
:100F10004D45F7D308F10100B0428046E4DB206A7A
:100F2000384420622046FFF7C9FEBDE8FF9F00005D
:100F3000625100002DE9F0418046D21D22F00702E7
:100F40000025D2E90002F52915A614D0011E72F180
:100F5000000106DA0023D0EB030063EB020211A6C6
:100F600008E0D8F800108B0701D50FA602E049076A
:100F700001D50EA601251146002408F1240704E03E
:100F800000F0D4F830323A55641C50EA0102F7D12F
:100F90002B46324621464046BDE8F041FFF7B1BE40
:100FA000000000002D0000002B00000020000000C9
:100FB00010B5002000F01AF8FFF780F9BDE81040E6
:100FC000012002F089BC10B5044602E0641C02F066
:100FD00085FC20780028F9D110BD0000004870473A
:100FE00020000020007B00F08000704710B500F06A
:100FF000F3FDBDE8104000F0EABD0000FEE7000090
:10100000C13F0008A54B0008394C0008D14B00082F
:101010004D4C0008254B000830B4002100F1240499
:1010200008E002F00705D208303542EA4372DB08D7
:101030006554491C52EA0305F3D10468002310A249
:10104000250708D504F020040C4304D0C46901230B
:101050000CA2641EC46130BCFFF753BE10B5044639
:1010600021461068FFF744FE02462046BDE81040C6
:101070000023D1E7D21D22F00701D1E90023CBE7FD
:1010800000000000300000002DE9F04791460F46B7
:1010900080460446002614F8015B2DB1FFF742F9A3
:1010A0000068405DC007F6D12B2D02D02D2D18D041
:1010B000641E4A463946204600F020FC27B13968B4
:1010C000A14201D1C7F800804FF0020471050BD591
:1010D0004042002803DDFFF789FD0460A007BDE85A
:1010E000F08746F48066E4E70028F8DAFFF77EFD33
:1010F00004606FF00040F2E7034640688C46002829
:1011000018BF88423CBF03464068F8D318681844AB
:10111000884207D00CF1030020F00700001D411A9F
:10112000521A0146081D0A60FFF733B930B5B0F115
:101130000A0271F100034FEA900E4EEA817EB0EB95
:101140000E0061EB91014FEA101E4EEA017E10EB9A
:101150000E0041EB11114FEA102E4EEA016E10EB1A
:101160000E0041EB11214FEA104E4EEA014E10EBFA
:101170000E0041EB1141401841F100014FEAD0004F
:1011800040EA41704FEAD1014FEA810444EA907489
:1011900010EB800544EB01046D1944EB0404521B71
:1011A000A3414FF0000348BF0A3200D530BD401CB8
:1011B00041F1000130BD2DE9FF4F0C461E464FF0B6
:1011C000FF378BB0D2E90001DDF860800A908A46D3
:1011D000C1F30A5505B93D46002108464FF000000D
:1011E000BAF1000F00F4400005DA00EB80004FF484
:1011F000400101EA50004FEA9059B9F1010F00DDBA
:10120000B9460A9850EA4A000ED044F61050A5F2AA
:10121000FF3545432F14B8F1000F1ED07542291E2B
:101220001EDDC9F100021CE0B8F1010F4FF0000013
:1012300001D0302103E0F24305E02154401CB042CC
:10124000FBDB30460022002121540B99C1F80880B5
:10125000C1E900200FB0BDE8F08FBD1B6D1CDEE7BB
:101260004A4600DA694206A800F036FC06AB93E86D
:10127000070003AB83E8070050460A9904F074FAAC
:101280008DE80700A0F500501F3800900398002D4E
:101290000ADD42F21F014A460844002303A90390D5
:1012A000684604F0DDFC09E0A0F500504A461F380E
:1012B000002303A90390684604F0E7FC8DE80700CB
:1012C0000004000C03D04FF0FF30410800E010464E
:1012D000B8F1000F03D00022009215461EE0751EE3
:1012E00005D4FFF723FF303262556D1EF9D5B346A2
:1012F0000122084302D000227F1C04E0207830281D
:1013000001D100227F1E002A099784D01DE0112DF3
:1013100007DAFFF70BFF303262556D1C50EA01020D
:10132000F5D1084302D00098C8B10EE00021681E34
:1013300005E0235C625C63542254401E491C8142D8
:10134000F7DBAB46A81B401E0990002004F80B00F9
:101350000B98099AC0F80880C0E9002B7AE711269B
:101360004FF0000857E72DE9F04F88460446D21D9C
:1013700022F0070191B0D1E90001CDE90A0104F0A2
:10138000BBFD02460B98C00F01D02D2007E020685E
:10139000810701D52B2002E0202101EAC000032AA9
:1013A000099001D0072A05DB03464146204600F09C
:1013B00045FB0BE12078800601D5E06900E00620BE
:1013C000B8F1650F814606D0B8F1660F18D0B8F1B4
:1013D000670F70D131E00020B9F1110F009001DBEF
:1013E000112301E009F101030AAA01A90CA8FFF7E2
:1013F000E2FEDDE90C70002609F10105834647E0B5
:1014000001204B4600904FF000470AAA01A90CA802
:10141000FFF7D1FEDDE90DB00C995D46002610B94D
:1014200009F101000D18B9EB050003D4C0F1FF3636
:1014300009F10105A5EB09002BE0B9F1010F01DA73
:101440004FF001090020B9F1110F0090484601DD6D
:10145000112300E003460AAA01A90CA8FFF7ABFE7E
:10146000DDE90C704D4600268346207800070AD43B
:10147000AB4500DA5D4601A8012D04DD411911F8E4
:10148000011C302907D04F4502DA17F1040F04DAA6
:10149000012082460FE06D1EEEE7002F02DCED1BFF
:1014A0003E4403E0781CA84200DD7D1CB81B00F11F
:1014B000010A4FF000472078000703D4AA4501DB5A
:1014C0004FF0FF3A0021B7F1004F0DF143088DF8BE
:1014D000431024D002202B23002F01DA7F422D233A
:1014E0000A21021EA0F1010000DC5FB197FBF1FCB4
:1014F00097FBF1F201FB1C7C17460CF1300C08F84D
:1015000001CDEEE7A8F1010003702188090501D59E
:10151000452100E06521A0F1010800F8011C0998AF
:101520000FA9A1EB0807FF1D00B10120411901EB34
:10153000EA70A1693844081A401EA0612078C006EC
:1015400002D42046FFF7A4FB099828B1D4E9012171
:101550009047206A401C20622078C00622D5204691
:10156000FFF796FB1EE0002E04DBB34502DD01A869
:10157000805D00E03020D4E901219047206A401CC2
:101580002062761CAAF101005FEA000A0AD1FFF787
:1015900029FBC0680168405CD4E901219047206ABA
:1015A000401C2062281EA5F10105DCDC07E0D4E91F
:1015B000012118F8010B9047206A401C2062381E58
:1015C000A7F10107F3DC2046FFF778FB032011B0F9
:1015D00041E600002DE9F04F04460D46D21D22F0F1
:1015E000070089B0D0E900974846394604F084FCEA
:1015F0000246F80F01D02D2307E02068810701D5AE
:101600002B2302E0202101EAC0038DF820300BB12A
:10161000012000E00020032A824601D0072A04DBD3
:101620002946204600F00AFA3FE12078800601D4DE
:101630000D2500E0E569C7F30A560D2D49DA0021B2
:101640004FEA175B08464FF00000002F00F44000FF
:1016500007DA00EB80004FF4400100EBD07001EAA4
:1016600060008115012901DD4FF0FF3100224FEAB2
:10167000850CBCF1180F06D31346ACF118004FF0DF
:101680008052C24003E04FF4801323FA0CF30CF1B4
:101690000C0CBCF1200F04D3ACF1200C09FA0CF0B7
:1016A00001E007FA0CF000294FF0004801DD18B9FD
:1016B0000FE00ED140450CD319EB02095F4121B96F
:1016C000404502D19F4329EA0209BBEB175F00D0D6
:1016D000761C2088000502D57B48784402E07A48D1
:1016E0007844193808AA302302F80A30037C0AF13A
:1016F0000101002E0AF1020A53546A4602DC4FF03F
:10170000300101E04FF031014FF001088DF8001079
:1017100002D0A6F2FF3603E059EA470100D06B4E33
:10172000002D02DC2178090704D54FF002082E2194
:101730008DF80110C44600210BE0C7F303433F01BD
:10174000C35C491C6D1E02F80830052908F1010828
:1017500001DA002DF1DC00210CE000EB1973491CCB
:101760001B786D1E082902F808304FEA091908F1A4
:10177000010801DA002DF0DC21688B0602D516E0A5
:10178000A8F10108E04505DD02EB080313F8013C70
:10179000302BF5D0B8F1000F09DD02EB080313F888
:1017A000013C2E2B03D1090701D4A8F10108002D1B
:1017B00005DD3E2102F808106D1E08F10108407C8D
:1017C000002E02F8080008F1010804DA2D20764204
:1017D00002F8080002E02B2002F808000A214FF46A
:1017E0007A70864208F101080BDB96FBF0F3303388
:1017F00002F8083096FBF0F308F1010800FB1366CD
:1018000001E0642E0CDB642096FBF0F3303302F829
:10181000083096FBF0F308F1010800FB136601E0C5
:101820000A2E06DB96FBF1F0303002F8080008F1D2
:10183000010896FBF1F001FB1060303002F808005F
:10184000A16908F1010808EB050202EB0A00081A79
:10185000A0612078C00602D42046FFF719FA216A59
:1018600008AE01EB0A00206204E0D4E9012116F879
:10187000010B9047BAF1010AF7D22078C00602D5D1
:101880002046FFF705FA6E4609E016F8010B3E28E0
:101890000FD0D4E901219047206A401C2062B8F1A2
:1018A0000108F2D22046FFF709FA09B00320BDE88B
:1018B000F08F206A2844206203E0D4E9012130201F
:1018C00090476D1EEBD3F8E72949000002FCFFFFAB
:1018D00010B5436913B1AFF3008001E0FFF7CCFA14
:1018E000012010BD128800F1240182840022C284EC
:1018F0000122EDE711684FF0FF32E9E72DE9F05FD3
:10190000824615468B4600270AF10104B946007845
:10191000302801D09DB113E014F8010B012778287D
:1019200003D0582801D045B10AE00DB1102D07D1E0
:10193000002714F8010B102502E0082500E00A2515
:101940000026B0460EE005FB080005FB06F1012766
:101950001FFA80F801EB1046B6F5803F00D3B94678
:1019600014F8010B294600F0A9F80028EBDABBF1C6
:10197000000F05D00FB1641E00E05446CBF80040C4
:10198000B9F1000F06D0FFF731F902210160C81E3E
:10199000BDE8F09F48EA0640FAE72DE9F041164617
:1019A0000C460546FEF7BEFC036893F801010128CA
:1019B00007D0FF2C12D8185D80B101202C70BDE833
:1019C000F081D3F807013246214603F20713C71806
:1019D0002846BC46BDE8F041002360474FF0FF3089
:1019E000EDE710B500F010F9BDE8104000F0EFB8D9
:1019F0007546FFF7F3FAAE4605006946534620F0F8
:101A00000700854618B020B5FEF778FCBDE82040F9
:101A10004FF000064FF000074FF000084FF0000BAA
:101A2000AC46ACE8C009ACE8C009ACE8C009ACE819
:101A3000C00921F007018D46704700002DE9F041F3
:101A40001F46044603260168072A01F4006004DBF0
:101A500008B116A505E016A503E008B115A500E03C
:101A600015A521F010002060A069C01EA0610FB173
:101A7000401EA0612046FFF70BF94FB1D4E90121C8
:101A800038469047206A401C2062C01C206206E055
:101A9000206AFAE7D4E9012115F8010B9047761E78
:101AA000F8D22046FFF70AF9BDE8F0814E414E001A
:101AB0006E616E00494E4600696E66003A2800D29B
:101AC000303820F02002412A01D3A2F137008842A9
:101AD00001D34FF0FF3070472DE9F047814616469D
:101AE0008AB0354878440DC88DE80D0032487844F6
:101AF000801C03AC0DC884E80D0041F69B300844FF
:101B0000372190FBF1F290FBF1F5A5F1800501FB87
:101B100012041B3C02D56442012000E00020DFF8E3
:101B200098A080460027FA44AAF1BE0A0EE0E0071A
:101B30000AD03246684607EB470101230AEB8101D0
:101B400004F0A3F88DE8070064107F1C002CEED190
:101B5000194F7F44AE3F19E0E80715D007EB04109A
:101B60000DF1180A90E80E008AE80E00C068F042F5
:101B700001D1981908903246012306A903A804F060
:101B800084F803AB83E807006D10641C002DE3D1DB
:101B90004FF0010332466946B8F1000F03A802D0A6
:101BA00004F05EF801E004F070F8C9E90001C9F83A
:101BB00008200AB0BDE8F087B045000010B5044623
:101BC000AFF300802046BDE81040FEF782BB00283E
:101BD00001D001F081BE704710B5002102A000F0D5
:101BE0003BF8012010BD0000534947414252543A8E
:101BF0002041626E6F726D616C207465726D696EEA
:101C00006174696F6E00000010B5012805D00021D5
:101C100003A000F021F8012010BD09A1F8E70000A1
:101C200053494752544D454D3A204F7574206F66C5
:101C30002068656170206D656D6F7279000000002D
:101C40003A2048656170206D656D6F727920636F11
:101C5000727275707465640070B505460C460A2092
:101C600000E06D1C01F03AFE35B128780028F8D16B
:101C700002E0641C01F032FE14B120780028F8D193
:101C8000BDE870400A2001F029BE00007047000046
:101C900010B543F61044C4F2020402F0D7F92068EC
:101CA00040F004002060206840F48030206054F848
:101CB000040CC0030BD543F20000C4F200004AF646
:101CC000AA2100BF016054F8042CD203FAD4206882
:101CD00020F00400206002F0AFF9002010BD0000E9
:101CE000B0B543F610450446C4F2020502F0AEF961
:101CF000204602F0FDF955F8041CC00041F0F00147
:101D000045F8041C022129602968C0B208432860F4
:101D1000286840F48030286055F8040CC003FBD4D8
:101D2000286820F00200286055F8040C10F0F00F2D
:101D300007D055F8040C012440F0F00045F8040CDD
:101D400000E0002402F078F92046B0BD72B600BF72
:101D5000FEE7000070B5866D044600F029F994F89E
:101D60003510022925D105462068216C026822F031
:101D700016020260426922F08002426109B9A16C38
:101D800019B1016821F008010160016821F0010129
:101D9000016000BF20680068C0070ED000F008F99D
:101DA000401B0628F6D320206065032084F8350008
:101DB0000CE080206065012008E0E06D3F2101FA21
:101DC00000F0B060012084F835000020002184F884
:101DD000341070BD90F83510022909D1052180F822
:101DE00035100068016821F0010101600020704792
:101DF00080214165012070472DE9F04F83B000F14B
:101E00003E4202F1FF724FEAB22241F600470192D0
:101E1000C4F2020708224FF0010E00254FF0000A1D
:101E20004FF00008B84208BF072200920AE000BF46
:101E300008F101080AF1040AB8F1100F05F10205D2
:101E400000F0A4800C680EFA08FB14EA0B09EFD02E
:101E50004C6804F0030CACF1010EBEF1010F11D877
:101E60000322876802FA05F6CA68B743AA403A43D4
:101E700082604268C4F3001722EA0B0207FA08F7EF
:101E80003A434260BCF1030F1CD0C26803238E6842
:101E900003FA05F7BA4306FA05F73A43BCF1020F15
:101EA000C2600FD16FF0030202EA580202440AF046
:101EB0001C060F23176A03FA06F40B69A743B34005
:101EC0003B431362026803234F68AB409A4307F019
:101ED0000303AB401A4317F4403F4FF0010E02607A
:101EE000A6D0002243F644030292C4F202031A6809
:101EF00043F6004442F480421A601A68C4F20104B6
:101F000002F480420292029A28F003024FF6084B34
:101F10002244CFF6FF7B52F80B300AF00C070F2655
:101F2000BE4023EA060C019B009E072B38BF1E46CD
:101F300006FA07F747EA0C0342F80B30A2684B6831
:101F400042EA090743F60C4CDE0258BF22EA0907B1
:101F5000A760C4F2010CDCF800209E0242EA0907E7
:101F600058BF22EA0907CCF8007062689E0342EA73
:101F7000090758BF22EA090767602268DB0342EAC3
:101F8000090358BF22EA0903236051E703B0BDE803
:101F9000F08F0000426902EA0103914341EA0341E4
:101FA00081617047002A08BF090481617047000001
:101FB00041F22850C2F200000068704740F2080069
:101FC00041F22851C2F20000C2F2000100780A6812
:101FD000104408607047000080B543F60040C4F22A
:101FE0000200016841F400710160016841F4806100
:101FF0000160016841F480710160032000F060F825
:102000000F2000F005F800F02BF8002080BD000044
:10201000B0B540F20802C2F2000240F204011278A8
:10202000C2F200014FF47A730968B3FBF2F204467E
:10203000B1FBF2F1084600F0FBFA0F2C4FF001055E
:102040000CD858B94FF0FF3021460022002500F08F
:1020500027F840F20C00C2F2000004602846B0BD30
:1020600082B0002043F640010190C4F202014A68A8
:1020700042F480424A604A6802F480420192019A26
:102080000090086840F080500860086800F08050B8
:102090000090009802B0704780B501F0B5FB80BD9C
:1020A00070B514460D46064601F0BEFB2946224691
:1020B00001F05EF80146304601F0BEFB70BD000045
:1020C00080B501F0CBFB80BD2DE9F041002800F088
:1020D0008B8043F60808C4F202080446D8F8F803D7
:1020E0000D4600F00700884207D288F8F853D8F868
:1020F000F80300F00700A84276D12068810717D5C1
:10210000410705D5D8F8001041F4E051C8F8001097
:10211000010705D5D8F8001041F46041C8F8001057
:10212000D8F80010A26821F0F0011143C8F800109F
:10213000C0073FD1D8F8F80300F00700A84207D93C
:1021400088F8F853D8F8F80300F00700A8424BD1FC
:102150002068410707D5D8F80010E26821F4E05163
:102160001143C8F80010000708D5D8F8000021690D
:1021700020F4604040EAC100C8F8000000F07EF89A
:10218000D8F8001046F2D002C1F30311C0F60002E5
:10219000515C40F2040220FA01F140F20C00C2F25C
:1021A00000000068C2F200021160FFF731FF00205A
:1021B000BDE8F0816068811E022907D258F8081C2A
:1021C00089015CBF0120BDE8F08110E0012807D142
:1021D00058F8081C89035CBF0120BDE8F08106E0C7
:1021E00058F8081C890702D40120BDE8F081D8F80E
:1021F000001021F003010843C8F80000FFF7D8FEE3
:10220000064641F2883700BFD8F80000616800F048
:102210000C00B0EB810F8DD0FFF7CAFE801BB842D7
:10222000F2D90320BDE8F08140F20400C2F20000C0
:102230000068704780B5FFF7F7FF43F60801C4F266
:102240000201096846F2E002C1F38221C0F60002F1
:10225000515CC84080BD000080B5FFF7E5FF43F644
:102260000801C4F20201096846F2E002C1F34231FA
:10227000C0F60002515CC84080BD000010B543F6B6
:102280000404C4F20204606800F00C0142F2004051
:102290000829C0F2F40007D0042918BF10BD41F28C
:1022A0000020C0F27A0010BD216801F03F022168D1
:1022B00023684902C3F3881105D4A1FB0001002360
:1022C000FEF78EF806E041F20020C0F27A004843A3
:1022D000B0FBF2F021680222C1F3014102EB41019F
:1022E000B0FBF1F010BD00002DE9F04182B00028F4
:1022F00000F0A2800446007843F60006C007C4F24E
:10230000020643D0B06800F00C00042805D1306804
:1023100080033BD56068C8BB8EE0B06800F00C005D
:10232000082802D170684002F1D46568B5F5A02F85
:102330000AD0B5F5803F0BD0306820F48030306093
:10234000306820F4802006E0306840F4802030605F
:10235000306840F480303060FFF72AFE002D0546DB
:1023600011D000BF3068800310D4FFF721FE401B5E
:102370006428F7D922E100BFFFF71AFE401B64284A
:102380004FF0030055D830688003F5D420788007DB
:102390001AD5B06810F00C0F09D0B06800F00C002E
:1023A000082840F08A807068400200F1868030681A
:1023B000800702D5E06801283ED13068216920F00D
:1023C000F80040EAC10030602078000738D4207857
:1023D00040074CD4A5695DB3B06800F00C00082834
:1023E00040F09E80012D27D07068E16900F48002E2
:1023F0008A4221D1216A00F03F028A421CD147F66D
:10240000C071626A0140B1EB821F15D1A26A00233C
:10241000CFF6FF7303EBC23200F440316FF30F02CB
:10242000914209D1E16A00F07060B0EB016F03D115
:10243000002002B0BDE8F081012002B0BDE8F081CB
:102440006069002840F20000C4F2472057D0012103
:10245000C0F8801EFFF7ACFD054600BF706F800717
:10246000B5D4FFF7A5FD401B0228F7D9A6E0306CD4
:1024700010F080580AD100200190306C40F080505C
:102480003064306C00F080500190019847F20007F2
:10249000C4F200073868C00524D4386840F480705E
:1024A0003860FFF785FD05463868C0051AD4FFF788
:1024B0007FFD401B0228F7D980E0E068002851D05A
:1024C0000020C4F2472001210160FFF771FD05469D
:1024D000306880073FF571AFFFF76AFD401B0228A7
:1024E000F6D96BE0A568052D50D0012D52D0306F84
:1024F00020F001003067306F20F004004DE0002133
:10250000C0F8801EFFF754FD054600BF706F8007BE
:102510007FF55DAFFFF74CFD401B0228F6D94DE07B
:102520000027C4F2472700203866FFF741FD022D3F
:1025300005460BD13068800158D5FFF739FD401BA7
:1025400002284FF00300F5D973E700BF306880011F
:102550007FF56EAFFFF72CFD401B02284FF0030004
:10256000F4D966E70020C4F2472000210160FFF79C
:102570001FFD0546306880077FF526AFFFF718FD81
:10258000401B02284FF00300F4D952E7306F40F0AF
:1025900004003067306F40F001003067FFF708FD3E
:1025A000002D054641F2883714D000BF306F8007F8
:1025B00013D4FFF7FDFC401BB842F7D9032002B04B
:1025C000BDE8F081FFF7F4FC401BB8424FF0030078
:1025D0003FF62FAF306F8007F4D4B8F1000F7FF4CF
:1025E000F9AE306C20F080503064F3E604F11C0545
:1025F0002FCD08430021CFF6FF7140EA821001EB96
:10260000C3316FF30F0140EA056008437060012099
:102610003866FFF7CDFC0446306880013FF508AF0F
:10262000FFF7C6FC001B02284FF00300F4D900E7B7
:1026300080B500F0F1FD80BD7047000070470000DC
:1026400010B590F83C20012A4FF0020252D001232D
:1026500080F83C3080F83D200268D2F804E0D2F8DF
:1026600008C00C682EF07003234341F2FF74C4F2DB
:102670000004A24253600DDC40F2FF73C4F2000379
:102680009A4215DCB2F1804F29D040F20043C4F2E7
:10269000000322E040F2FF33C4F201039A4212DC4D
:1026A00041F60003C4F200039A4218D0002312E05E
:1026B00040F60003C4F200039A4210D040F60043F3
:1026C000C4F2000309E044F20003C4F201039A4299
:1026D00005D040F20043C4F201039A4204D1496894
:1026E0002CF08003194391600121002280F83D10F5
:1026F00080F83C20104610BD002804BF0120704720
:1027000010B5044690F83D0028B9002084F83C003C
:10271000204600F01FF8022084F83D002068211DAB
:1027200000F0FAFD012084F8460084F83E0084F8A9
:102730003F0084F8400084F8410084F8420084F8A7
:10274000430084F8440084F8450084F83D000020EC
:1027500010BD000080B582B0006840F20041C4F2B4
:102760000001884201D002B080BD0020019043F6F4
:102770004000C4F202000168002241F00201016041
:102780000068002100F00200019001981D20FFF771
:1027900087FC1D20FFF780FC02B080BD90F83D1043
:1027A00001291CBF01207047022180F83D100068FC
:1027B00041F2FF72C168C4F20002904241F001018F
:1027C000C1600DDC40F2FF71C4F20001884215DCEB
:1027D000B0F1804F29D040F20041C4F2000122E064
:1027E00040F2FF31C4F20101884212DC41F60001DF
:1027F000C4F20001884218D0002112E040F6000126
:10280000C4F20001884210D040F60041C4F2000139
:1028100009E044F20001C4F20101884205D040F20F
:102820000041C4F20101884206D1816801F007012C
:10283000062904BF00207047016841F001010160D2
:102840000020704710B5044690F83C0001284FF076
:10285000020008BF10BD012284F83C2084F83D002E
:1028600020684FF6777382689A4382600A684F2A1D
:102870000FDC1F2A22DD202A23D0302A21D0402A33
:102880004DD14B68CA68194600F0F0FD2068402120
:102890003BE06F2A17DDB2F5005F20D0B2F5805F14
:1028A0002AD0702A3BD1D1E9012CCB68614600F0D7
:1028B000C9FD2068816841F077011AE00AB1102A49
:1028C0002DD1114621E0502A18D0602A27D14B681B
:1028D000CA68194600F0DCFD2068602115E0D1E9E6
:1028E000012CCB68614600F0ADFD2068816841F4A1
:1028F0008041816000200BE0002009E04B68CA683D
:10290000194600F0B3FD2068502100F0A7FD00201B
:10291000012184F83D10002184F83C1010BD0120F5
:10292000F6E7000070470000B0B504460068C168D3
:10293000026902EA0105A9071DD4680731D42807F6
:1029400047D4E8065CD4E80773D128067BD4680630
:1029500006D520686FF040010161204600F0A4F820
:10296000A80658BFB0BD20686FF020010161204665
:10297000FFF764FEB0BD6FF0020101610121217714
:102980008069800703D02046FFF7CCFF05E0204692
:1029900000F064F8204600F063F800202077680714
:1029A000CDD520686FF00401016102212177806993
:1029B00010F4407F03D02046FFF7B4FF05E0204627
:1029C00000F04CF8204600F04BF800202077280754
:1029D000B7D520686FF00801016104212177C06933
:1029E000800703D02046FFF79DFF05E0204600F05A
:1029F00035F8204600F034F800202077E806A2D50C
:102A000020686FF01001016108212177C06910F47E
:102A1000407F03D02046FFF785FF05E0204600F009
:102A20001DF8204600F01CF800202077E8073FF44E
:102A30008CAF20686FF001010161204600F012F8B0
:102A400028067FF584AF20686FF080010161204681
:102A5000FFF7F2FD68067FF583AF7AE77047000065
:102A60007047000080B5016840F20040C4F20000E9
:102A7000814200D080BD40F2800CC2F2000CBCF854
:102A800000204CF6CD41CCF6CC415143531CB1F162
:102A9000333FACF8003088BF80BD00F500308021A6
:102AA000FFF778FA80BD0000704700007047000013
:102AB00070470000B0B582B0036804461868D96852
:102AC0005A6900F02F05202D01F0200505D125B110
:102AD000204600F02BFD02B0B0BD5FEA007C1EBFB7
:102AE00002F0010E01F4907212EB0E024AD1226B39
:102AF0000840C1063DD5012A3BD10020019018684D
:102B000001905868019001985869400642D4A08D00
:102B1000E18DE28D002A1CBF401A5FEA004101D11D
:102B200002B0B0BD216851E8031F226821F4907102
:102B300042E80313002BF5D1216851E8051F2268F4
:102B400021F0010142E80513002BF5D1202184F882
:102B500042100021216300BF216851E8031F226851
:102B600021F0100142E80313002BF5D1022161632B
:102B700054E0010654D44006D2D5204600F0CAFCE9
:102B800002B0B0BDC20718BF11F480725DD1420718
:102B900061D467E0E06B016849688AB2002A44D0DA
:102BA000A38D9A4241D2E185C069B0F5807F30D0D3
:102BB000206850E8030F216820F4807041E8030288
:102BC000002AF5D1206850E8050F216820F00100A7
:102BD00041E80502002AF5D1206850E8050F216878
:102BE00020F0400041E80502002AF5D1202084F8B9
:102BF00042000020206300BF206850E8030F2168D6
:102C000020F0100041E80302002AF5D1E06BFFF745
:102C1000A1F802206063A08DE18D401A81B20FE01F
:102C2000204600F06FFD02B0B0BDA18D91427FF44F
:102C300077AFC069B0F5807F7FF472AF0220606328
:102C40002046FFF733FF02B0B0BD626C42F00102D4
:102C50006264420706D5BEF1000F03D0626C42F0F9
:102C600002026264820706D5BEF1000F03D0626CD7
:102C700042F004026264BCF1000F06D55EEA050270
:102C800003D0626C42F008026264626C002A3FF476
:102C900047AF0840800602D5204600F047FC206878
:102CA0004069616C00F0400001F00801401827D035
:102CB000204600F007FC2068406940061BD500BF95
:102CC000206850E8050F216820F0400041E8050227
:102CD000002AF5D1E06B70B143F2B541C0F60001B6
:102CE0000165FFF777F800283FF41AAFE06B016D3C
:102CF000884702B0B0BD2046FFF7DAFE02B0B0BD93
:102D00002046FFF7D5FE0020606402B0B0BD000091
:102D1000002804BF0120704710B5044690F8410018
:102D200028B9002084F84000204600F021F8242033
:102D300084F841002068C16821F40051C160204638
:102D400000F058FC2068016921F49041016141695B
:102D500021F02A014161C16841F40051C1600020A5
:102D60002021606484F8411084F84210606310BD33
:102D700010B586B0006844F20042C4F2000200219F
:102D80009042CDE90411CDE90211019126D041F222
:102D90000001C4F20101884253D1002043F6300102
:102DA0000090C4F202014A69252442F010024A61EF
:102DB0004A6902F010020092009A0090086840F000
:102DC00001000860086800F00100009000984FF4CE
:102DD000C06001900020C4F202001FE043F6300002
:102DE0000091C4F202000269262442F4003202611A
:102DF000026902F400320092009A0091016841F0E9
:102E000008010160006800F0080000900098602050
:102E100001900020C4F2020000F5406002210291FE
:102E200000210391032104910721059101A9FEF7D7
:102E3000E3FF204600210022FFF732F92046FFF78A
:102E40002BF906B010BD000010B590F84230202BD1
:102E50001CBF022010BD00294FF0010418BF002A3A
:102E600001D1204610BD0024046300F031FC20464F
:102E700010BD00002DE9F04381B0044640F2D810A7
:102E8000C2F2000041F240488442C2F2000808D079
:102E900008F1240120460122FFF7D6FF01B0BDE86A
:102EA000F0830CA508F12409474602E0FF69002FD2
:102EB000EED0002FECD0BE69002EF7D03846294660
:102EC000FDF736FE0028F1D1786949460122B04766
:102ED000ECE700BF7369675F756172745F73696760
:102EE000000000002DE9F041044690F84100202840
:102EF0001CBF0220BDE8F0810E4600294FF0010002
:102F000042D01746002A08BFBDE8F0814FF0000804
:102F100021201D46C4F8448084F84100FFF748F89A
:102F2000A784E784A1680746B1F5805F0DD12069C9
:102F3000002814BF3046B046064606E016F8010BDE
:102F400021684860E08C0138E084E08C80B1204644
:102F500080213A462B4600F0FFFBB8B9002EEDD198
:102F600038F8020B21686FF35F2048600026E9E71C
:102F7000204640213A462B4600F0EEFB202184F803
:102F80004110002818BF0320BDE8F081202084F8FC
:102F900041000320BDE8F08170470000FEE700001B
:102FA0000020704770B586B0002543F630000595C7
:102FB000CDE90355CDE901550095C4F20200016841
:102FC00040F2004441F0800101600168C4F2020453
:102FD00001F080010091009900950168002241F004
:102FE000010101600168802601F001010091009952
:102FF0000095016841F008010160016801F00801D5
:10300000009100990095016841F00201016000689B
:10301000802100F00200009000982046FEF7C2FFD9
:103020000120CDE9020501A9204601960495FEF78D
:10303000E3FE06B070BD000080B586B040F24810D7
:1030400040F200420021C2F20000C4F20002C72395
:1030500042F2CF0CCDE90411CDE90211CDE9001106
:10306000C0E90023C0E9021C01618161FFF744FB54
:10307000002818BFFEF76AFE4FF48050029040F21D
:103080004810C2F2000002A9FFF7DCFB002818BFBD
:10309000FEF75CFE0020CDE9000040F24810C2F2CD
:1030A00000006946FFF7CCFA002818BFFEF74EFE75
:1030B00040F24810C2F20000FFF770FB06B080BD7E
:1030C00080B540F2901041F20001C2F20000C4F25B
:1030D000010100234FF00C0C4FF4E13280E80E00A8
:1030E000C0E90333C0E905C3C361FFF711FE00283F
:1030F00018BFFEF72BFE41F24040C2F2000000F183
:10310000240140F29010C2F200000122FFF79CFE61
:1031100080BD000080B540F2D81044F20041C2F2F8
:103120000000C4F2000100234FF00C0C4FF4E13218
:1031300080E80E00C0E90333C0E905C3C361FFF7AF
:10314000E7FD002818BFFEF701FE41F24040C2F241
:10315000000000F1240140F2D810C2F20000012268
:10316000FFF772FE80BD0000FEE70000FEE70000F2
:1031700000F0070080F00703042B28BF04234FF062
:10318000FF3C03380CFA03F338BF00209943814019
:103190000CFA00F022EA0000084370477047000074
:1031A000F0B581B043F60C4714460E460546C4F20E
:1031B000020700F04BFFF01C396820F0030041F0DB
:1031C000F001002639607E60F8B140F2012100BFB5
:1031D0007A680A437A6022682A6000BF3A68D2039C
:1031E000FCD47A6822F001027A603A6812F0F00F9B
:1031F00006D10435043804F10404E9D1002604E0C2
:103200003868012640F0F000386000F015FF3046C5
:1032100001B0F0BD70470000B0B501380024B4EB38
:10322000106F1CBF0120B0BD4EF21005CEF200059C
:1032300068604FF0FF300F2100F0FEFA0720AC600D
:1032400028602046B0BD000080B5FEF7B7FE80BD07
:1032500070B592B006AC20463021FDF73FFC00254A
:1032600043F640000595CDE90355CDE9015500959C
:10327000C4F202000168022641F08051016000683A
:1032800000F080500090009847F200000095C4F2D2
:103290000000016841F4804101600068A82100F449
:1032A000804000900098012006904FF480300790F5
:1032B0004FF480000D9004200E90119020460C9643
:1032C000CDE90F16FFF710F888B90F20CDE90106F8
:1032D0004FF4A05004904FF48050059001A80521B0
:1032E0000395FEF7F1FE002804BF12B070BDFEF793
:1032F0002DFD00004EF68850CEF20000016841F42A
:10330000700101607047000080B540F24810C2F2C1
:103310000000FFF709FB80BDB0B540F6FF3E056831
:10332000C4F2000E40F2004C7045C4F2010C0FDCF8
:10333000B0F1804F19D040F20043C4F2000398422C
:1033400013D040F60003C4F2000398420DD011E000
:1033500040F60043C4F20003984206D0604504D012
:103360000023C4F20103984204D14B6825F0700297
:1033700043EA020541F6FF73C4F2000398420DDCF4
:1033800070451FDCB0F1804F41D040F20043C4F2E1
:10339000000398423BD040F6000321E043F6FF7360
:1033A000C4F20103984220DC42F20003C4F200039D
:1033B00098422CD00023C4F20103984227D06045E4
:1033C00025D029E040F60043C4F2000398421ED005
:1033D00041F60003C4F20003984218D041F60043BE
:1033E000C4F20003984212D016E044F20003C4F283
:1033F000010398420BD044F60003C4F20103984243
:1034000005D044F20043C4F20103984204D1CB68D2
:1034100025F4407243EA02050A688C684B69C4626D
:1034200040F480648262644504BF096901630268F4
:1034300025F0800142F0040219430260012242613A
:103440000160B0BDD0F808C011432CF47F4C41EAB4
:10345000032141EA0C01816070470000826822F07C
:103460007002114341F0070181607047D0F820C01D
:10347000036A23F001030362836923F0F00343EA44
:1034800002122CF00A0319438261016270470000A6
:10349000D0F820C0036A23F010030362836923F489
:1034A000704343EA02322CF0A00343EA0111826127
:1034B0000162704780B5806B0021C185FFF7F8FA83
:1034C00080BD0000016851E8031F026821F490717B
:1034D00042E80313002BF5D1016851E8051F02688B
:1034E00021F0010142E80513002BF5D1016B012900
:1034F0000AD100BF016851E8031F026821F01001E2
:1035000042E80313002BF5D1202180F8421000215E
:103510000163704780B50168CA6822F04002CA6042
:10352000202180F84110FFF737FD80BD80B582B0C3
:1035300090F8421022291ED18268B2F5805F02D134
:10354000016900294AD0816AB2F5805F07D00AB9C3
:10355000026922B10268526802F07F0201E002684B
:1035600052680A700121826A11448162C18D013959
:103570000A04C18501D002B080BD0168CA6822F08A
:103580002002CA60CA6822F48072CA604A6922F0C6
:1035900001024A61202180F8421000214163026B40
:1035A000012A23D1016300BF016851E8031F0268AB
:1035B00021F0100142E80313002BF5D101680A68DD
:1035C000D20606D5002201920A680192496801914B
:1035D0000199818DFFF76AFA02B080BD0168826AA5
:1035E00049686FF35F2111800221BCE7FFF742FCBD
:1035F00002B080BD10B504460068D4E902C2236958
:10360000016921F4405111430161626943EA0C01EF
:10361000E3691143C268194349F20C639A431143A9
:10362000C1604169A26921F4407141F20043114334
:1036300040F48062C4F201039A42416102D1FEF774
:103640000BFE01E0FEF7F6FDE16963681922B1F5B2
:10365000004FA0FB02011CD15A00DB0FFCF7C0FE9B
:1036600048F21F51C5F2EB11A0FB01235A096FF07C
:10367000630302FB0300322303EBC000A0FB010144
:103680004FF4F87000EA111000EB0210C1F3421180
:103690001AE09A009B0FFCF7A3FE48F21F51C5F2F7
:1036A000EB11A0FB01235A096FF0630302FB030037
:1036B000322303EB0010A0FB0101F02000EA5110BF
:1036C00000EB0210C1F3431122680843906010BD63
:1036D000816200218285C2854164222180F84210E6
:1036E000016921B10168CA6842F48072CA60016848
:1036F000486940F001004861C86840F0200200209D
:10370000CA60704790F84110212923D18168B1F532
:10371000805F01D1016931B1016A02684B1C03620B
:103720000978516007E0016A036831F8022B6FF3F2
:103730005F225A600162C18C01390A04C18418BF3A
:1037400070470068C16821F08001C160C16841F024
:103750004001C160704700002DE9F04182B004468D
:10376000006800680840884203D1002002B0BDE82C
:10377000F0811D460E4690465F1C04E020680068FC
:103780003040B04228D0002FF8D0FEF711FC01469F
:103790004FF003000DB3A1EB0801A9421DD820682A
:1037A000C1684907EAD5402EE8D0802EE6D00168EE
:1037B0000907E3D500250195016801914068019052
:1037C00001982046FFF77EFE0820606484F8405090
:1037D000012002B0BDE8F081002002B0BDE8F08118
:1037E00080B540F29010C2F20000FFF763F980BD8F
:1037F00080B540F2D810C2F20000FFF75BF980BD3F
:1038000000207047FEE70000002848BF704700F026
:103810001F01012202FA01F14EF200124009CEF21C
:10382000000242F8201070474EF60C50CEF2000015
:103830000068C0F3022070474EF6145300F00F02E8
:10384000CEF2000309011A4400F16043B0F1FF3FDA
:10385000C8BF03F564421170704700004EF60C516A
:10386000CEF200010A684FF6FF031A4060F30A2205
:1038700042F0806040F0FD700860704780B50369D9
:10388000984780BD80B5C368984780BD8068704701
:10389000808870478180704780B5D0F82031002B38
:1038A0000CBF0020984780BD80B5D0F82431002B94
:1038B00018BF984780BD000080B5D0F82431002B98
:1038C00018BF984780BD000080B54369984780BD08
:1038D00080B58369984780BD70470000704700003D
:1038E00000284FF0000218BF002901D11046704790
:1038F000826822B18A4208D01268002AFAD182680E
:10390000C0E9011101200A6070470022104670478B
:10391000B0B540F28804C2F200042046C021FDF791
:10392000DDF84FF6C055C0F6090505F5C070C02199
:1039300001F0F8F841F26841C2F200012846C022C5
:1039400001F084F905F5E07004F14001402201F036
:103950007DF9B0BD70B598B30446006803282FD830
:10396000DFE800F00286143A00200125208104F1EE
:10397000180080212560FDF7B1F86068D4F89C102C
:103980000860D4F89800056002202060206904F1E6
:103990000C054368667B2946012298479EB10028A2
:1039A00000F0968028780A2800F08E80202811D018
:1039B0000D2800F0898000202060042040B270BDF6
:1039C000FF2040B270BD002800F0828028780028D7
:1039D0007AD02075032020602069617B436839B369
:1039E00004F10C05294601229847002870D0287858
:1039F000202813D12189B4F90A2000202073881AC5
:103A0000D4F8981020440A68D4F89C301830561C1A
:103A100043F822004FF6FF700E6060812089217B01
:103A200022180130208160891176013060811DE00B
:103A300004F1160102229847002849D02069218903
:103A4000436804F11805E28A2944984700283FD0CA
:103A5000D4F8981020890B682A185D1C0D60E18A43
:103A6000D4F89C60084446F823202081012020607F
:103A7000607BF8B1207B0A2804D00D2802D0208971
:103A80007F28A7D3D4F898602189B4F90A20356833
:103A900004F118038A1AD4F89CE00139002003EBE2
:103AA000020C6A1C218189B2207332604EF825C055
:103AB00058540AE0D4F89800217D0068884203DC5D
:103AC00020897F28FFF486AF0020206040B270BDBF
:103AD00000202060012040B270BD000080B5844607
:103AE00000284FF0000005D00029CCF8000018BFD6
:103AF000002A00D180BD002BFCD0DDF808E0BEF12B
:103B0000000F08BF80BD0398CCF8102000228CF86D
:103B10000D006046CCE90112CCE9263E80BD0000D4
:103B200010B558B104460068022812D001280AD006
:103B300020B9012020600020208102E0FF2040B257
:103B400010BD0120206060682189405CA8B102207E
:103B50002060E06804F10A0143680122984780B1BF
:103B6000218962684B1C2381A07A515C8842E8D08D
:103B700000202060042040B210BD0020206040B230
:103B800010BD00202060012040B210BD0346002877
:103B90004FF0000008BF7047002918601FBF002ABF
:103BA0005960DA601846704710B548B3044600689B
:103BB000022815D0012805D010BBA168012020766D
:103BC000C4E900016068F0B1E06800F051FC616890
:103BD000887B18B1E068898900F06AFC02202060C7
:103BE0006068D0E90110884705281CD0C0B20428BD
:103BF00025D0012832D100202076012040B210BD0E
:103C0000FF2040B210BD207E90B3E06804F119019E
:103C1000012200F041F8A06850B3002181810068C2
:103C20000028FBD124E0E06800F03AFAA06870B107
:103C3000002100BF818100680028FBD107E0606897
:103C4000807B20B1E06800F081FA6168888160685B
:103C500001680120C4E9000140B210BDE06800F035
:103C60001FFAA06820B10021818100680028FBD1E3
:103C70000020206040B210BD4FF0000248B1026049
:103C800039B144F21D32C0F60002C0E903114261AD
:103C90007047002070470000F0B581B090B10E462B
:103CA000F9B10546EFF3108072B61446E9882A8907
:103CB000914201D1698909B1297C11B380F310883F
:103CC00000244FE046F2E41046F2EB2146F2F922DE
:103CD000C0F60000C0F60001C0F60002FCF712FCBE
:103CE000FEE746F2E41046F2CC2146F2F922C0F695
:103CF0000000C0F60001C0F60002FCF703FC00BFA4
:103D0000FEE70121297480F31088EF88EFF310801B
:103D100072B66989AA88EB88A142A2EB030238BF78
:103D20000C46A242D8BF53421A19091BEA80698186
:103D3000AA81E98180F31088A888C21B2868A24262
:103D400000EB070108DA3046FCF72FFEA888296847
:103D5000C21BB018A21A01E030462246FCF725FE2D
:103D600000202874204601B0F0BD00002DE9F0418C
:103D7000054600284FF0000058D00C46002955D0C9
:103D80001646002A52D09846002B08BFBDE8F081A5
:103D9000E86948B92420FCF7CDFA98B324210746F6
:103DA000FCF79CFEEF613D62EF6921463846FCF767
:103DB000BFFE18B13846FCF7D9FD60B32420FCF7EC
:103DC000B9FAE8B124210546FCF788FE38462146B9
:103DD000FCF7AEFE28B97869B04202D1B869404517
:103DE0000ED097B1F86980B121460746FCF7A0FED6
:103DF0000028F7D17869B042F4D1B8694045F1D1D3
:103E0000002040B90020BDE8F081FD612F62012053
:103E10002F460028F6D02046C7E90568FCF7A6FD26
:103E2000024638462146FCF7C0FD0120BDE8F0817E
:103E30002DE9F04381B0A0B10E4611B30546EFF372
:103E4000108072B61446E9882A89914203D16989A3
:103E500009B1697C09B1297C19B380F31088002469
:103E60006EE046F2E41046F2EB2146F20732C0F66D
:103E70000000C0F60001C0F60002FCF743FB00BFE3
:103E8000FEE746F2E41046F2CC2146F20732C0F6D5
:103E90000000C0F60001C0F60002FCF733FB00BFD3
:103EA000FEE70121297480F31088B5F80880EFF34C
:103EB000108E72B6A9886A89A142A1EB020338BFAD
:103EC0000C46A34215DA6F7C97B1B5F80690E31A59
:103ED0001FFA83FCA1EB0900271A6045A2EB03003F
:103EE000C8BF09EB0307EF806881AF81E88100E07C
:103EF0001C462889A7B2091AB942D8BF4842698925
:103F0000204428810819E98968810819E8818EF31D
:103F10001088A888A0EB08022868BA42404409DA51
:103F20003146FCF742FDA9882868A1EB0802B118C8
:103F3000BA1A01E031463A46FCF737FD00202874F2
:103F4000A0B201B0BDE8F083B0B54FF68064C0F612
:103F5000090400F0B7FE18BB40F28805C2F2000564
:103F600004F1C0002946C02200F032FED5F88000DE
:103F7000B0B1286C002804BF286810F1010018D0E7
:103F80000421C0F60201086800F07F40B0F1006F24
:103F900018BFB0BD51F8040C096800F089F9B0BD34
:103FA00041F26841C2F200012046C02200F010FE3A
:103FB000B0BD41F26841A4F1C000C2F20001F4E7D3
:103FC00010B582B04FF6806401460020C0F60904A7
:103FD00001902046C02200F039FE04F5A07001A92E
:103FE000042200F033FE02B010BD000010B540F214
:103FF0008804C2F200042046C021FCF76FFD4FF692
:104000004070C0F609002146402200F01FFE10BD9E
:1040100046F2C811C0F6000109684A6A824208D80F
:10402000896A1144814282BF46F2C810C0F600007E
:10403000704700207047000043F61040C4F20200B1
:10404000016841F0004101607047000043F6004004
:1040500040F22311C4F20200C4F26751416048F6F5
:10406000AB11CCF6EF514160016801F00F01016026
:10407000C16841F0F001C1607047000010B582B026
:1040800004468DF8070040F2D810C2F200000DF18E
:10409000070101226423FEF725FF204602B010BD70
:1040A00080B548B1EFF3108172B68289C389C280AE
:1040B000438181F3108880BD46F2E41046F2EB2183
:1040C000C0F60000C0F6000102A2FCF71BFA00BF18
:1040D000FEE700BF6765745F616C6C5F7065656B60
:1040E0006564000080B5006800F01EF980BD000026
:1040F00070B50646FFF78CFF01684FF0000C486A68
:10410000D1E91035CC6C321A002008E0661C03D1CE
:104110008E6AB54228BF70BD0130FF2813D0AA4275
:104120001D4401D3AA420FD3A542EFD38E6AB542F4
:10413000ECD20CF1010C5FFA8CF301EBC306D6E96B
:104140001035F46CE2E7FF2070BD000080B550B17F
:10415000EFF3108172B68289C3889A420FD28088A9
:10416000D21A10440CE046F2E41046F2EB21C0F6FD
:104170000000C0F6000104A2FCF7C4F9FEE7D01A63
:1041800081F3108880B280BD6765745F7065656B70
:104190005F73746174757300002818BF1030704726
:1041A00080B5FDF705FF002180BD000082B0FDF75E
:1041B00013FFFFF74DF8FEF7F5FEFEF781FFFEF760
:1041C0003BFFFEF7A7FF2CA0FCF72AFB40F640655B
:1041D000C2F2000540F22021C2F2000128464FF44D
:1041E0000062002300F008F940F62064C2F20004E7
:1041F00020462946FFF740FD2046FFF7CDFF41F25C
:10420000A036C2F200060146304600F0C3FD20464B
:104210003146FFF765FB46F2B000C0F60000D0E97A
:10422000000140F65867C2F20007CDE90001694677
:10423000384600F0ABFA20463946FFF751FB41F211
:10424000404043F63163C2F2000010A1C0F6000303
:104250002A46FFF78BFD40F2D81244F6A14306F13F
:1042600078000EA1C2F20002C0F60003FFF77EFD47
:104270002046FFF799FCFBE70D0A4E41495F426F6C
:104280006F745F56302E310D000000007369675F58
:10429000756172745F736967000000007369675F1E
:1042A000796D6F64656D5F7265635F736967000048
:1042B000002282F31488BFF36F8F8546084770474A
:1042C00070B50DA000F0CCFA46F25430C0F60000F4
:1042D00046F26C36A0F10C050CA4C0F6000600BF37
:1042E00055F80C1F2046AA6800F0BAFA05F10C0038
:1042F000B042F5D1002070BD0D0A7368656C6C206A
:10430000636F6D6D616E64733A0D0A00252D313651
:1043100073202D2025730D0A0000000080B5006871
:1043200000F002F880BD0000F0B581B090B10E46FB
:10433000F9B10546EFF3108072B61446A9892A89AF
:10434000914201D1E98909B1297C11B380F3108828
:1043500000244DE046F2E41046F2EB2146F2DA2268
:10436000C0F60000C0F60001C0F60002FCF7CAF873
:10437000FEE746F2E41046F2CC2146F2DA22C0F61D
:104380000000C0F60001C0F60002FCF7BBF800BF59
:10439000FEE70121297480F31088AF89EFF31080C4
:1043A00072B6E989AA88AB89A142A2EB030238BFA1
:1043B0000C46A242D8BF53421A19091BAA81E981AF
:1043C00080F31088A888C21B2868A24200EB07016E
:1043D00008DA3046FCF7E9FAA8882968C21BB01849
:1043E000A21A01E030462246FCF7DFFA00202874CA
:1043F000204601B0F0BD000080B538B100294FF073
:10440000000C18BF002A0ED1604680BD46F2E410B1
:1044100046F2EB21C0F60000C0F600010BA2FCF74B
:1044200071F800BFFEE7EFF3108C72B60160002157
:104430008280C0F80610C0F80A10C181437401746C
:104440008CF310888446604680BD00BF7175657529
:10445000655F696E69745F62797465004EF60C5130
:104460000422CEF20001C0F2FA5200200A60704726
:1044700080B548B1EFF3108172B6C288438982815A
:10448000C38181F3108880BD46F2E41046F2EB212F
:10449000C0F60000C0F6000102A2FCF733F800BF2E
:1044A000FEE700BF72657365745F7065656B000041
:1044B00080B590B1EFF3108C72B6C38882880B443C
:1044C0009A1A38BF1A46C38982818B4298BF0B461D
:1044D000591AC1818CF3108880BD46F2E41046F26F
:1044E000EB21C0F60000C0F6000102A2FCF70AF8BA
:1044F000FEE700BF726573746F72655F7065656B10
:104500005F7374617475730010B582B078B104463E
:104510000068032839D8DFE800F002860C52012039
:10452000206084F8C5000020A4F8C2007BE0FF20D2
:1045300095E0201DFFF7F4FA042828D0C0B2012826
:1045400029D0A8BB0020A4464CF8C80F3CF8061C94
:104550005CF8143CCCE90100CCE90300CCE905008F
:10456000CCF81C0001EB41015CF80C2C53F8211035
:104570001CF804ECACF1B4000CF12003CDE900CE42
:10458000FFF7ACFA0B2003210FE0FF2067E0B4F83F
:10459000C200013005E0B4F8C210002084F8C50064
:1045A000481CA4F8C20003200121216018B955E07D
:1045B0000020002852D0032835D00B284FD104F119
:1045C0001400FFF7C7F9042814D0C0B2012817D08F
:1045D00030BBB4F8C200D4F8B42000EB400102EBC9
:1045E0008101D4F8E8004A6804F1C801904701202D
:1045F00000210FE0B4F8C2000130A4F8C20007E0C7
:10460000B4F8C2000130A4F8C200002084F8C5004C
:10461000032001212160032805D0F8B100201EE00D
:1046200000200328F9D1B4F8C200D4E92D1200EB20
:10463000400001EB8000904209D00168D4F8BC2012
:10464000201DFFF7A3FA02202060012007E094F864
:10465000C5000021216008B1042000E0012040B223
:1046600002B010BD844600284FF0000005D0002A9B
:10467000CCF8000018BF002900D17047002B08BFFC
:1046800070470098CCF8B4108CF8C4006046CCF8A1
:10469000B820CCF8BC30704710B582B00446043066
:1046A000FFF732FF042808D0C0B201280DD080B92E
:1046B00004F1F000FFF7F4FC0BE004F1F0000DF161
:1046C00007010122FFF7E8FA03E004F1F000FFF729
:1046D000CFFE204600F0A0F902B010BD40F63C60CD
:1046E000C2F200000068704740F63C61C2F200016F
:1046F00008607047B0B50D460446FBF713FE01682D
:1047000094F83301095C202910D011F099010DD1E2
:104710005E2806DCA0F12D01022907D3082805D068
:10472000B0BD7F2802D05F2818BFB0BD28780C2804
:104730000CDC082818D00A280CD0B4F82C01294623
:104740000130A4F82C012046012216E07F280BD06E
:104750000D28F2D1002046F20321A4F82C01C0F666
:10476000000120460C2208E0B4F82C0138B10138D1
:10477000A4F82C0104A120460322FFF795F800209D
:1047800084F83301B0BD00BF08200800F0B581B047
:10479000E9B30446002846D044F2996004F11005BC
:1047A000C0F6000000220127C4E90020A560A28114
:1047B000A773D1E9000104F58076C4E94C0104F542
:1047C000A271304680220123FFF716FE44F2E50075
:1047D000C0F6000046F2543146F26C3204F58A739A
:1047E000C4E9456004F11400C0F60001C0F60002FF
:1047F0000097FFF737FF2846FFF776FF46F20320C2
:10480000C0F6000000F02CF8204601B0F0BD46F2E2
:10481000E41046F21022C0F600000DA1C0F600021E
:10482000FBF770FEFEE746F2E41046F21022C0F6F7
:10483000000003A1C0F60002FBF764FEFEE700BF24
:104840004E554C4C20213D2070744F626A00000090
:104850004E554C4C20213D2070744F707300000069
:1048600083B070B581B0054605A80EC0FFF736FFCE
:10487000F8B10446EFF3108072B694F8321111B11A
:1048800080F3108815E0012184F8321104F50D76CB
:1048900080F3108805AB304680212A460093FBF751
:1048A00017FE82B220463146FFF706F8002084F852
:1048B000320101B0BDE8704003B070472DE9F0430C
:1048C00081B0B0F82A510446002D4FD0B4F83071B1
:1048D000052F28D304F2B44904F5DA784846414656
:1048E0008022FBF7F3FF002840D004F52D70042749
:1048F00000F1800631468022FCF79CF8013F3046EB
:10490000F6D1C5F1800109EB05007F2D88BF00219C
:10491000FCF7C2F8484641462A46FCF78BF80520CA
:10492000A4F8300122E04FB104EBC71000F50D7080
:1049300004F5DA718022FBF7C9FFB8B104EBC710A8
:1049400000F52D76C5F180017019A4F82E7104F5DB
:10495000DA787F2D88BF0021FCF79EF8304641466B
:104960002A46FCF767F8781CA4F83001B4F8300147
:10497000A4F82E0101B0BDE8F0830000B0B540F608
:104980002060C2F2000014460D46FFF705FC4368A4
:10499000294622469847B0BD70B5044600780228E3
:1049A00027D00D4601280ED000281CBF012070BD65
:1049B0000126C4F80260FFF7F3FB0A3041F1000161
:1049C000C4E902012670A1886288A4F58870294490
:1049D000FEF762FF6188814203D10021002021702F
:1049E00070BD20B1A2880244081AA2806080022013
:1049F0002070FFF7D5FBD4E90223801A71EB030086
:104A00004FF000014FF00500B8BF0121002918BF89
:104A10000120217070BD000070B5044604F233150A
:104A200000F588702946FFF7B7FF052828D0C0B2E7
:104A3000002864D12D780C2D28DC082D50D00A2DAB
:104A400028D0FBF76FFC0068405D20280AD010F0EA
:104A5000990007D1A5F12D00022803D35F2D1CBFBB
:104A6000042070BDB4F82A017E284AD8411C204495
:104A700080F8B4510120A4F82A11A4F8281170BDBF
:104A800020462946FFF736FE052070BD7F2D27D032
:104A90000D2DD6D104F5DA75B4F82A612846FBF756
:104AA00065FFA6B1B04212D12046FFF707FFB4F868
:104AB0002A0194F83311421C2044A4F82A2180F8DA
:104AC000B41104F1F00092B22946FFF7B1F928467B
:104AD0008021FCF703F80020A4F82A01012070BD12
:104AE000B4F82A0158B10138A4F82A0114FA80F167
:104AF0000022A4F82801012081F8B42170BD012012
:104B000070BD0020C4F82801012070BD10B540F22E
:104B1000D810C2F2000064231446FEF7E3F92046E1
:104B200010BD00002DE9F04381B089460646FFF72D
:104B30006FFA90B3EFF3108872B607460068A9F1D8
:104B40000101806A002481420BD388F3108825E09C
:104B50001020396801EBC000006C04444C45064449
:104B6000F3D239690029F0D0304688470028ECD1CB
:104B70003968002003E000BF01301028E8D001EBC5
:104B8000C002936C0133E4D04B6AD56CF31AAB428C
:104B9000F2D2526C9342EFD3DBE70024204601B0FF
:104BA000BDE8F083B0B5054680071CBF0020B0BD4E
:104BB0002846FFF72DFA044620B1636828460021F5
:104BC00000229847002C18BF01242046B0BD0000E9
:104BD000F0B581B014460E460546FFF719FAEFF31B
:104BE000108772B610B3A90701D000241EE0016837
:104BF0002A19D1E90931D21A8A4201D9002415E0D3
:104C000083693BB12846214632469847002818BFA1
:104C100000240BE054B1701E002100BF15F8012BD9
:104C200001318BB2A34200F8012FF7D387F310882C
:104C3000204601B0F0BD000010B50446FFF7E8F9CA
:104C400010B1816820468847012010BD2DE9F04150
:104C5000144688460746FFF7DBF9EFF3108672B675
:104C60000028254618BF002515D017F0030112D1E2
:104C70000168E219D1E90931D21A8A4201D9002525
:104C800009E04369002533B138462146424698473A
:104C9000002808BF254686F310882846BDE8F08125
:104CA00040F2D813C2F20003984218BF704780B593
:104CB00040F2D810C2F200006423FEF713F9BDE8F9
:104CC0008040704700207047B0B50022012918DBF2
:104CD00041F2210E03788C46013982EA032208232F
:104CE00014B28EEA4205B4F1FF3FA3F10103C8BF3D
:104CF00055001A062A46F3D1BCF1020F00F101005B
:104D0000E8DA90B2B0BD000010B578B1D1B10022A0
:104D1000027091E80C50D1E9044142608360C0F810
:104D20000CC0C0F810E0C0E9054110BD46F2A22059
:104D300046F23D21C0F60000C0F6000140F262429A
:104D4000FBF784FD46F23D2103A0C0F6000140F2CE
:104D50006342FBF77BFD00BF4E554C4C20213D20AC
:104D600070744F707300000080B500F0A3F807283E
:104D70000CD80121814011F0230F01D040B280BD39
:104D800011F0C00F1EBF042040B280BD002040B211
:104D900080BD0000B0B586B0F8B1044644F6695253
:104DA000C0F600020023A16446F2B801C4E9003253
:104DB0000122C0F60001A381A27391E80C50D1E951
:104DC00004511030CDE904516946A0608DE80C50C3
:104DD000FFF79AFF204606B0B0BD46F2EB2046F240
:104DE0003931C0F60000C0F600017B22FBF72EFD32
:104DF00080B518B1806B4368984780BD46F2EB20C0
:104E000046F23931C0F60000C0F600015622FBF729
:104E10001DFD0000F0B581B0002840D006460446D4
:104E200016F82809022824D00D4601280DD098BB79
:104E300000201F46A0806280FFF7B2F9C01941F13F
:104E40000001C4E9020101202070A08862882918AD
:104E50003046FEF739FD6188814202D102200021EF
:104E600017E020B1A2880244081AA28060800220C4
:104E70002070FFF795F9D4E90223801A71EB030043
:104E80004FF000014FF00500B8BF0121002918BF05
:104E90000120217001B0F0BD012001B0F0BD46F24B
:104EA000A22046F23D21C0F60000C0F600017D229E
:104EB000FBF7CCFC70B5002800F043810446007875
:104EC000092800F23681DFE810F00A000D00170013
:104ED000A400B500BF000C012B012B007E0044F2A2
:104EE00001302060611C20460122FEF7F1FC002801
:104EF00000F01F810220207004F11C00002100F04E
:104F000037F9811E08291FD805460120DFE801F086
:104F10001E1C1C3605051C1C0500022876D108E164
:104F2000651C04F128002946012240F6B833FFF73A
:104F300071FF052829D002283BD1287804283AD1CE
:104F400009202070002038E0022014E0A0680078DA
:104F500068B12046FEF79CFC05462046FEF796FC0D
:104F6000014620462A46FEF78DFC85423AD140F2A2
:104F7000036020800020022848D1DAE00020207061
:104F800005250120022841D1D3E046F21B2046F23C
:104F9000B12146F23D22C0F60000C0F60001C0F685
:104FA000000240F25123FBF7ADFA002005252070E6
:104FB00002E0022001E006250120022800F0B9806D
:104FC000012800F0AB800620214601F8010F2046A1
:104FD0000122FEF77DFC002800F0AB8000200125B7
:104FE00020709BE046F21B2046F23D22C0F60000F6
:104FF0005AA1C0F600024FF4CF73FBF783FA0020EA
:1050000020700B250120022800F09380012800F079
:105010008580611C20460122FEF75AFC002800F022
:105020008880A068007830B3E0780130E07044F206
:1050300004302080611C20460122FEF749FC002834
:1050400000F0778005202070E17804F11C0000F06A
:105050008FF8421E0B2A40D80021DFE802F04010F2
:105060002B310640400633063E29A0780130C1B2FC
:10507000A07015202BE00025E8B2257070BD2046F9
:10508000FEF704FC06462046FEF702FC02462046D8
:105090003146FEF7F3FB06462046FEF7F9FB864253
:1050A00006D1E0780130E0700620A4F8010012E09B
:1050B00018200FE041F207502080012000210EE06F
:1050C000062007E0A0780130C1B2A07006200929AF
:1050D00088BF1820607006202070012128460546F0
:1050E000E1B1651C204629460122FEF7F1FBB8B16B
:1050F0002878182820D146F21B2046F2BE2146F21D
:105100003D22C0F60000C0F60001C0F6000240F2E9
:105110002F23FBF7F7F9002004250FE0E8B270BD5C
:10512000611C20460122FEF7D3FB00281CBF08208B
:1051300020700125E8B270BD052002252070E8B27C
:1051400070BD46F2A22046F23D21C0F60000C0F636
:1051500000014FF4BD72FBF779FB00BF696E636F0E
:10516000727265637420646174612073697A65008A
:105170002DE9F04381B0002800F066810646044620
:1051800016F81C09072800F201818846DFE810F0B4
:1051900008000A0050006E009800C600E1001B01E4
:1051A00001202070A71C04F10C003946012240F6B2
:1051B000B833FFF72FFE05282DD0022831D13878DB
:1051C0004FF00609421E172A4FF001002AD880210D
:1051D000DFE812F01A00180028002E01280028002D
:1051E000280028002800280028002800280028007F
:1051F000280028002800280028002800280028006F
:10520000280034014FF480613046FEF743FB022052
:105210002070002006E0002020704FF005090120DA
:1052200000E00220022800F0B180002840F0B080A9
:1052300004F10C00E11C01224FF47A73FFF7EAFD40
:10524000022806D005280AD14FF0050901200021C7
:1052500001E0002003212170022804D196E0022001
:10526000022800F09380002840F0928004F10C00A6
:10527000211D01224FF47A730125FFF7CBFD05288C
:1052800013D0022817D1E07821794840B0F1FF050A
:1052900018BF0125FF38B0FA80F04FEA50104FEAEE
:1052A000800118BF4FF0070901E0002181462170FD
:1052B000022D03D16AE00225022D67D0002D67D1AF
:1052C000304604F10C07FEF7E1FA05463046FEF7DA
:1052D000DFFA02463846294642F21073FFF79AFD7C
:1052E000052810D0022815D13046FEF7CFFA054622
:1052F0003046FEF7CDFA01462846FFF7E5FC0021CF
:105300000522208102E0012100228146227002292B
:1053100003D13BE00221022938D0C9BB04F10C00C3
:10532000611D01224FF47A73FFF774FD022806D045
:1053300005280AD14FF005090120002101E00020D5
:1053400006212170022803D120E0022002281DD06E
:10535000F0B904F10C00A11D01224FF47A7301256C
:10536000FFF758FD05280BD002280CD1B4F8050032
:105370002189000400BA88420FD1002507211DE0D1
:10538000002181461AE00225022D1AD14FF00109B1
:105390005FFA89F001B0BDE8F08346F21B2046F2C7
:1053A0003D22C0F600002EA1C0F600024FF4A0730B
:1053B000FBF7A8F84FF00A09012500212170022D02
:1053C000E4D0002DE4D1E078404503D0A8F10101FC
:1053D00081421BD1A8F10101814211D146F21B206B
:1053E00046F23D22C0F6000028A1C0F6000240F2BD
:1053F0005713FBF787F8002020704FF00909C7E723
:105400000020207020814FF00209C1E746F21B20E6
:1054100046F23D22C0F6000016A1C0F600024FF48D
:10542000B173FBF76FF8002020704FF00809AFE769
:10543000002020704FF003090120F3E600202070C7
:105440004FF004090120EDE646F2A22046F23D218C
:10545000C0F60000C0F60001B822FBF7F7F900BF64
:10546000696E636F727265637420636865636B6FE6
:1054700075740000696E636F727265637420706189
:10548000636B6574206E756D626572006475706C17
:105490006963617465207061636B6574206E756DFE
:1054A000626572002DE9F04381B000284DD00546B9
:1054B0000F46D0E9180140F20009C0F60209461A69
:1054C0001446964228BF164601EB0900394632467B
:1054D000FFF7BCFB81B2B14223D138463146FFF71A
:1054E000F3FB696E804601EB090039463246FFF74F
:1054F0006FFB81B2B14219D138463146FFF7E4FB68
:10550000804518D1D5E9180131448142696618D126
:10551000FEF76CFD46F21530C0F60000FBF780F98F
:105520000FE00FA0FAF7EEFF00240AE016A0FAF74A
:10553000E9FF002405E002461EA04146FAF7E2FF1B
:105540000024204601B0BDE8F08346F2EB2046F28D
:105550003931C0F60000C0F600012A22FBF776F9C7
:1055600074617267657420666C6173682077726914
:1055700074652064617461206572726F722E2030D0
:105580007825782E0D0A00007461726765742066B4
:105590006C61736820775265616453697A65206431
:1055A000617461206572726F722E20307825782EBA
:1055B0000D0A0000436865636B206572726F722E7E
:1055C000205772697465436865636B3A3078257853
:1055D0002052656164436865636B3A307825782EA4
:1055E0000D0A0000F0B581B0C0B30546002005F1FA
:1055F0003C076866384614460E46FBF793F9FBF7FE
:10560000B5F930440130E865FBF7FCF8286619A0CD
:105610003946FAF777FF296E1CA0FAF773FF296E57
:10562000B1F5002F04D92DA0FBF7FAF8002412E001
:105630000020C0F60200FFF775FA2A6E904204D2ED
:105640001FA0FBF7EDF8002405E0014615A0FAF7CE
:1056500059FFFEF75DF9204601B0F0BD46F2EB20A0
:1056600046F23931C0F60000C0F600010D22FBF70A
:10567000EDF800BF596D6F64656D2066696C655FFC
:105680006E616D653A2573200D0A0000596D6F64D7
:10569000656D2066696C655F73697A653A2564207B
:1056A0000D0A0000666C6173682065726173652085
:1056B000737563636573733A2564200D0A000000F7
:1056C00074617267657420666C61736820657261CD
:1056D0007365206572726F722E200D0066696C65AD
:1056E0002073697A65206F757472616E67652066D4
:1056F0006C6173682073697A652E200D00000000CC
:105700002DE9F041D0B11446884600F1680611A792
:1057100002E000BFF66976B16EB1B569002DF9D02F
:1057200030463946FBF704FA0028F3D17069414648
:105730002246A847EEE72046BDE8F08146F2EB207E
:1057400046F23931C0F60000C0F600015D22FBF7D9
:105750007DF800BF7369675F796D6F64656D5F7217
:1057600065635F73696700005FEA400C08BF91F0F2
:10577000000F4FEA8C234FEAC12243EA51514FEA0E
:105780001C5018BF00F5F0404FEA300018BF41F040
:1057900000415FEA6C5C00F02980BCF1FF3F08BF6C
:1057A00040F080407047130C06BF12044FF0100CFD
:1057B0004FF0000C130E04BF12020CF1080C130F73
:1057C00004BF12010CF1040C930F04BF92000CF102
:1057D000020CD30F04BF52000CF1010C11464FF024
:1057E0000002A0F11F00A0EB0C00704711F0004F69
:1057F00008BF704731F000413FF4D5AF0B0C06BF36
:1058000009044FF0100C4FF0000C0B0E04BF0902FE
:105810000CF1080C0B0F04BF09010CF1040C8B0FE9
:1058200004BF89000CF1020CCB0F04BF49000CF13E
:10583000010CCCF1200322FA03F341EA030102FA3E
:105840000CF2A0EB0C0000F10100704723F07F4741
:1058500020F07F4C80EA030000F00040ACEB07032F
:1058600003F57C5303F1FF032DE9804909B44FEAA6
:10587000144324EA03484FEA154B25EA0B4E0FF276
:10588000042606EB13273E7803FB0667C7F50007DF
:1058900007FB06F64FEAD64606F102064FEA5437F2
:1058A00007FB066CCCF1005C4FEA1C472CEA074C66
:1058B0000CFB06F507FB06F404EB15464FEA9616BB
:1058C00049085FEA320234BF00204FF000404FEA3F
:1058D000D13706FB07FC4FEA1C4C0CFB0BF7D21B25
:1058E00003FB0CF761EB07010CFB0EF7B0EB074075
:1058F00072EB17420CFB08F734BFA2EB0742B2EB86
:10590000074261EB17414FEA0C444FEA910706FB4F
:1059100007FC4FEA1C4C0CFB0BF7B0EBC74072EBDB
:10592000573203FB0CF734BFA2EBC742B2EBC742BE
:1059300061EB57310CFB0EF7B0EBC70072EB5772FF
:105940000CFB08F734BFA2EBC702B2EBC70261EB56
:1059500057714FEA816141EA92114FEA826242EA4D
:1059600090124FEA806004EBCC04039F4FEAD137DA
:1059700006FB07FC4FEA1C4C0CFB0BF7D21B03FB8E
:105980000CF761EB07010CFB0EF7B0EB074072EB75
:1059900017420CFB08F734BFA2EB0742B2EB0742F9
:1059A00061EB17414FEA8C5504EB9C244FEA9107B9
:1059B00006FB07FC4FEA1C4C0CFB0BF7B0EBC74097
:1059C00072EB573203FB0CF734BFA2EBC742B2EBCA
:1059D000C74261EB57310CFB0EF7B0EBC70072EB1F
:1059E00057720CFB08F734BFA2EBC702B2EBC70239
:1059F00061EB57714FEA816141EA92114FEA82628D
:105A000042EA90124FEA806015EB4C2544F1000405
:105A10004FEAD13706FB07FC4FEA1C4C0CFB0BF797
:105A2000D21B03FB0CF761EB07010CFB0EF7B0EB8D
:105A3000074072EB17420CFB08F734BFA2EB07429A
:105A4000B2EB074261EB17414FEA813141EA9241E3
:105A50004FEA823242EA90424FEA80304FEA0C76B7
:105A600015EB1C1544F1000448EA03434EEA0B48C9
:105A70004FF0000EB2EB080C71EB030724BF624637
:105A800039464EEB0E0E4FF0000B001852414941C3
:105A90004BEB0B0BB2EB080C71EB03077BF1000B2C
:105AA00024BF624639464EEB0E0E4FF0000B001835
:105AB000524149414BEB0B0BB2EB080C71EB030766
:105AC0007BF1000B24BF624639464EEB0E0E51EAC5
:105AD000020718BF46F0010616EB0E7655F10002DC
:105AE00054F1000103D5BDE88901BDE80088BDE897
:105AF0008901BDE80048B619524141EB0101A3F10B
:105B00000103704780807F7E7D7C7B7A7978777611
:105B100076757473727171706F6E6E6D6C6C6B6A8A
:105B20006A69686867666665646463636261616028
:105B3000605F5F5E5E5D5D5C5C5B5B5A5A595958A5
:105B4000585757565655555554545353525252510F
:105B5000515050504F4F4F4E4E4D4D4D4C4C4C4B65
:105B60004B4B4A4A4A4949494848484747474746AC
:105B700046464545454444444443434343424242E8
:105B8000424141419C46002B30D477002BD04FEA54
:105B900037071CB503B44FF010004FF01001BAF1F5
:105BA000000F06D0BCF1000FDCBF40F0080040F051
:105BB00008014FF000000FBCBDE810400BF1010BD5
:105BC000BBF1010F08BF5FEA170722BF12F1010204
:105BD00011F101014FF0004143F1000300F00040DA
:105BE00043EA00007047F9D35708D0E746EA064673
:105BF0004FEA164613F1400F1FDD13F1200FDFBFF0
:105C000016430A46002120335B42BED0C3F1200771
:105C100046EA06464FEA164602FA07F746EA07063C
:105C200022FA03F2C3F1200701FA07F742EA07025A
:105C300021FA03F14FF00003A7E746EA020646EA1D
:105C400006464FEA164646EA0106BCBF46EA064645
:105C5000360C4FF000034FF000024FF0000194E7C4
:105C60002DE9804C70B49A46934691E8380007C8F5
:105C700031EA400C48BF34EA430C03D5FFF7E6FD98
:105C8000FFF780FFF0BCBDE8008C2DE9804C70B4BC
:105C90009A46934691E8380007C810F0804F08BF35
:105CA00013F0804F03D100F005F8FFF76BFFF0BC55
:105CB000BDE8008C20F07F4723F07F4C80EA030092
:105CC00000F0004007EB0C03A3F57C53A3F1FE03A7
:105CD00092F0000F00F0B38095F0000F00F0778095
:105CE0002DE901494FEA114021EA00484FEA1446E4
:105CF00024EA064700FB06FC08FB06F607FB08F84B
:105D000018EB06484CEB164C00FB07F718EB07485E
:105D10004CEB17404FEA124B22EA0B4E4FEA154666
:105D200025EA06470BFB06FC0EFB06F607FB0EFEFC
:105D30001EEB064E4CEB164C0BFB07F71EEB074E0B
:105D40004CEB174B18EB0B0840F1000018EB0E0B57
:105D500058EB000840F100008F1A4FF000014FF09F
:105D600000063CBFC943661B14BFB5EB040C002101
:105D70003CBFC943F61B4FEA174427EA04454FEAE4
:105D80001C472CEA074C04FB076205FB07F70CFBDA
:105D900005F616EB074642EB174204FB0CFC16EB2C
:105DA0000C4642EB1C421BEB060658EB020241413B
:105DB0004EEA8E0E46EA9E0601D5BDE80189B61967
:105DC000524141EB0101A3F10103BDE801894FEA12
:105DD000144524EA05464FEA114721EA074C05FB22
:105DE00007F406FB07F70CFB06F111EB074144EB48
:105DF000174405FB0CFC11EB0C4144EB1C444FEA2F
:105E0000124722EA074C05FB07F206FB07F70CFBDB
:105E100006F616EB074642EB174205FB0CFC16EBA9
:105E20000C4642EB1C456A1854F1000148BF70470C
:105E3000B619524141EB0101A3F10103704795F0FE
:105E4000000F37D04FEA114221EA02464FEA1447C9
:105E500024EA074C02FB07F106FB07F70CFB06F4EC
:105E600014EB074441EB174102FB0CFC14EB0C4410
:105E700041EB1C414FEA154725EA074C02FB07F5A9
:105E800006FB07F70CFB06F616EB074645EB174536
:105E900002FB0CFC16EB0C4645EB1C42121951F1AF
:105EA000000148BF7047B619524141EB0101A3F10F
:105EB000010370474FEA144524EA05464FEA1147AB
:105EC00021EA074C05FB07F106FB07F70CFB06F27E
:105ED00012EB074241EB174105FB0CFC12EB0C42A5
:105EE00051EB1C414FF0000648BF7047921841EB40
:105EF0000101A3F10103704703B401984100009828
:105F000050EAC12018BF04204A0D18BF40F001001C
:105F100040F2FF72B2EB515F08BF40F0020001286F
:105F200008BF052002B0704730380A2801D201208E
:105F3000704700207047000010B500290AD008788B
:105F4000002807D005487844FAF7F2FD002801D070
:105F5000002010BD0248784410BD00004604000037
:105F60003E04000010B500290AD00878002807D0A8
:105F700005487844FAF7DCFD002801D0002010BD68
:105F80000248784410BD00002A05000022050000E8
:105F9000F1EE100A4FF6FF71C0F2C03120EA0100A5
:105FA00040F04070E1EE100A7047FBF7DCB9FBF7F8
:105FB00011BB3031323334353637383941424344FE
:105FC0004546403058003031323334353637383971
:105FD0006162636465664030780004000008000078
:105FE000000000000002000100001000000000009E
:105FF00000000000303132333435363738396162D1
:106000006364656678700030313233343536373842
:1060100039414243444546585000000002400000C8
:10602000000000A00000000005400000000000C8C3
:10603000000000000C4000000000409C0000000038
:10604000194000000020BCBE0000000034400000E9
:10605000BFC91B8E00000004B5400000504BCFD0DC
:106060006607E2CF010000006C4100003E8251AAA9
:10607000DFEEA73401000000D9420000DCB5A0E249
:106080003A301F97FFFFFFFFB4450000FD25A0C871
:10609000E9A3C14FFFFFFFFFFF3F000000000080AA
:1060A00000000000FF3F0000000000800000000032
:1060B0007D4900080D4B000800040000200A002064
:1060C000E5550008A5540008F14D000801570008E7
:1060D0000000000000000000010203040607080998
:1060E0000000000001020304010153544D33324605
:1060F00034787820314D4220466C6173680000008E
:106100000000000000000000000001000000000886
:10611000000010000004000000000000FF0000006C
:1061200064000000F40100000040000000000000D6
:106130000000010000000100000002000000020059
:10614000FFFFFFFFFFFFFFFF000000000000000057
:10615000000000000000000000000000000000003F
:10616000000000000000000000000000000000002F
:10617000000000000000000000000000000000001F
:10618000000000000000000000000000000000000F
:1061900000000000000000000000000000000000FF
:1061A00000000000000000007265626F6F740072F2
:1061B00065626F6F740068656C70007368656C6C05
:1061C0002068656C70000000E8600008A12F0008DE
:1061D00001380008911C0008E11C0008A1310008EA
:1061E0000000000028257329206861732061737303
:1061F000657274206661696C656420617420257322
:106200002E0A000D0A6B6B407368656C6C203E00B3
:106210007368656C6C5F696E6974000A4572726FB1
:10622000723A20257320696E2066696C652025739B
:10623000206174206C696E652025640A00453A2F40
:1062400055736572732F4C495A48454E4759414E14
:10625000472F417070446174612F4C6F63616C2FE4
:1062600041726D2F5061636B732F6B6B2F4D6963A0
:10627000726F426F6F742F302E392E372F736F75F8
:106280007263652F636F6D6D756E69636174696F9D
:106290006E2F796D6F64656D2F796D6F64656D2EEE
:1062A00063004E554C4C20213D2070745468697336
:1062B00000726561642074696D656F757400747235
:1062C0007920636F756E74206D6178004E554C4C6B
:1062D00020213D207044617465007065656B5F62CC
:1062E000797465735F7175657565004E554C4C200A
:1062F000213D2070744F626A006465717565756533
:106300005F627974657300656E71756575655F624E
:106310007974657300446F776E6C6F616420666991
:10632000726D7761726520746F20666C617368208E
:10633000737563636573732E005254452F4D696303
:10634000726F426F6F742F796D6F64656D5F6F74DC
:10635000612E6300A86100085D440008AF61000879
:10636000B6610008C1420008BB610008C0640008B3
:106370000000002020000000C4010008E0640008C4
:1063800020000020101B0000E001000810010000A8
:1063900043000000F8FFFFFF004040404040404005
:1063A00040404141414141404040404040404040E8
:1063B000404040404040404040050202020202028C
:1063C00002020202020202020220202020202020DB
:1063D00020202002020202020202909090909090EF
:1063E00010101010101010101010101010101010AD
:1063F0001010101002020202020288888888888821
:10640000080808080808080808080808080808080C
:106410000808080802020202400000000000000014
:10642000000000000000000000000000000000006C
:10643000000000000000000000000000000000005C
:10644000000000000000000000000000000000004C
:10645000000000000000000000000000000000003C
:10646000000000000000000000000000000000002C
:10647000000000000000000000000000000000001C
:10648000000000000000000000000000000000000C
:106490000000000000000000000000001C000000E0
:1064A00043000000F8FFFFFF0C0000000E0000009A
:1064B0000F0000002E00000091DAFFFF0000000036
:1064C000010000000024F4000100000010000000A2
:1064D00000000000000000000000000000000000BC
:040000050800018965
:00000001FF
